:100000000C9417060C9498280C94C5280C943F0661
:100010000C943F060C943F060C943F060C943F064C
:100020000C943F060C943F060C94B50C0C943F06C0
:100030000C943F060C943F060C943F060C943F062C
:100040000C94F2280C943F060C948A2C0C94C52C2A
:100050000C943F060C943F060C943F060C943F060C
:100060000C943F060C943F06E51BEC1BEC1BE51BB8
:10007000EC1BEC1BEC1BEC1BEC1BEC1BEC1BEC1B48
:10008000EC1BEC1BEC1BEC1BEC1B5A1BEC1BEC1BCA
:10009000EC1BEC1BEC1BBD1AEC1BEC1BEC1BEC1B58
:1000A000EC1BEC1BEC1BEC1BEC1BEC1BEC1BEC1B18
:1000B000EC1BEC1BEC1B661B661B661B661B661BA6
:1000C000661B661B661B661BEC1BEC1BEC1BEC1B10
:1000D000EC1BEC1BC21A651B651B651B651BEC1B2F
:1000E000761B7E1B861B8E1B961B9E1BA61BAE1BA8
:1000F000B81BC21BCC1BD61B091BC91AEC1BEC1B63
:10010000EC1BEC1B5A1BEC1BEC1BEC1BEC1BEC1B49
:10011000EC1BEC1BEC1B641B641B641B641BEC1BC7
:10012000761B7E1B861B8E1B961B9E1BA61BAE1B67
:10013000B81BC21BCC1BD61B091BC91AEC1BEC1B22
:10014000EC1BEC1B5A1B1D1C1D1C1D1C1D1C1D1C0F
:100150001D1C1D1C1D1C1D1C1D1C1D1C1D1C1D1CD7
:100160003D1D3D1D3D1D3D1D3D1D3D1D641C6E1C69
:10017000781C821CE81CF21C001D111DAE1D1E1EE9
:10018000EF1DF41DF91DFE1D031E081E0D1E1E1E73
:10019000181E2B2540254C255525622588259025A0
:1001A000B325A025456E746572206D656E752E2E83
:1001B0002E00546F67676C6564206D6963726F50C1
:1001C000504D00546F67676C656420696E76657288
:1001D0007465642050504D2100546F67676C6564EE
:1001E000205458206D7574696E672100546F6767DD
:1001F0006C65642074656C656D657472792100505E
:10020000726F746F636F6C206572726F72207769A2
:1002100074682052580054696D656F757420776852
:10022000656E20636F6E6E656374696E6720746FB0
:1002300020525800507265737320616E79206B658F
:100240007920746F2063616E63656C00436F6E6E1E
:10025000656374696E6720746F2052582C20706F2C
:100260007765722075702074686520525820287751
:100270006974682062696E6420706C7567206966B5
:10028000206E6F74207573696E6720616C77617979
:10029000732062696E642900546F67676C6564201F
:1002A00027696D6D656469617465206F757470751B
:1002B000742700546F67676C65642027736C6176E0
:1002C00065206D6F64652700546F67676C656420F7
:1002D00027616C776179732062696E642700546FBF
:1002E00067676C65642050504D206368616E6E6571
:1002F0006C206C696D6974005365742052535349C6
:1003000020696E6A656374696F6E206368616E6EE2
:10031000656C2028303D3D64697361626C6529001D
:100320005365742050504D206D696E696D756D2058
:1003300073796E630053657420626561636F6E202C
:10034000696E74657276616C0053657420626561D4
:10035000636F6E2064656C6179005365742062651B
:1003600061636F6E206672657175656E6379206971
:100370006E20487A3A20303D64697361626C652C66
:100380002050783D504D52206368616E6E656C2040
:10039000782C2046783D465253206368616E6E6526
:1003A0006C2078005365742050574D2073746F7023
:1003B0002064656C61792028302064697361626C07
:1003C00065642C20312D323535203D3D20302E31D5
:1003D00073202D2035306D696E29005365742050CF
:1003E000504D2073746F702064656C6179202830E3
:1003F0002064697361626C65642C20312D3235355F
:10040000203D3D20302E3173202D2035306D696E1A
:100410002900536574206661696C736166652064A8
:10042000656C61792028302064697361626C656451
:100430002C20312D323535203D3D20302E3173209A
:100440002D2035306D696E29002A2A2A2A2A2A2A67
:100450002A2A2A2A2A2A2A2A2A2A2A2A2A2A2A2AFC
:100460002A2A2A2A2A2A0052582041636B656420CE
:100470002D2072657665727420737563636573737E
:1004800066756C21002A2A2A2A2A2A2A2A2A2A2A36
:100490002A2A2A2A2A2A2A2A2A2A2A2A2A2A2A2ABC
:1004A0002A2A002A2A2A2A2A2A2A2A2A2A2A2A2AD6
:1004B0002A2A2A2A2A2A2A2A2A2A2A2A2A2A2A2A9C
:1004C0000052582041636B6564202D207570646173
:1004D0007465207375636365737366756C21002A98
:1004E0002A2A2A2A2A2A2A2A2A2A2A2A2A2A2A2A6C
:1004F0002A2A2A2A2A2A2A2A2A2A2A2A0056616CE1
:1005000069642063686F69636573206172653A206E
:100510005B315D2D5B31365D20286368616E6E65F1
:100520006C20312D31362900536574206F7574703D
:10053000757420666F7220706F727420005B585D56
:100540002061626F7274206368616E6765732061F9
:100550006E64206578697420525820636F6E6669F6
:1005600067005B535D207361766520736574746901
:100570006E677320746F205258005B525D20726565
:10058000766572742052582073657474696E67734F
:1005900020746F2064656661756C747300557365B3
:1005A000206E756D62657273205B312D445D207421
:1005B0006F206564697420706F727473205B452DC1
:1005C000515D20666F722073657474696E67730085
:1005D000202D20726563656976657220636F6E6693
:1005E0006967757261746F722C207278207377203E
:1005F000000A0A6F70656E4C52536E672000536597
:10060000742073657269616C2062617564726174D3
:10061000653A200056616C69642063686F696365A0
:10062000733A2031202D20342B34202F2032202DDE
:100630002038202F2033202D20382B34202F203419
:10064000202D203132202F2035202D2031322B3407
:10065000202F2036202D203136005365742043682A
:10066000616E6E656C20636F6E6669673A20005339
:1006700065742044617461726174652028302D3284
:10068000293A200053657420486F70206368616EBA
:100690006E656C7320286D61782032342C20736570
:1006A0007061726174656420627920636F6D6D6141
:1006B00073292076616C69642076616C756573209E
:1006C000312D3235353A2000536574206368616EF0
:1006D0006E656C2073706163696E672028783130B5
:1006E0006B487A293A200053657420524620706F77
:1006F0007765722028302D37293A20005365742001
:100700005246206D616769632028686578292065F5
:100710002E672E20307844454144463030443A20FC
:10072000005365742062617365206672657175653A
:100730006E63792028696E20487A293A20005B5A36
:100740005D20656E74657220726563656976657299
:1007500020636F6E66696775726174696F6E20756C
:1007600074696C79005B465D20646973706C6179B3
:100770002061637475616C206672657175656E6366
:100780006965732075736564005B525D2063616CFD
:1007900063756C6174652072616E646F6D206B654A
:1007A0007920616E6420686F70206C697374005BDF
:1007B000495D207265696E697469616C697A65204A
:1007C00073657474696E677320746F20736B6574DE
:1007D00063682064656661756C7473005B585D20A6
:1007E000726576657274206368616E6765732061F7
:1007F0006E642065786974206D656E75005B535D6D
:1008000020736176652073657474696E67732074F4
:100810006F20454550524F4D20616E6420657869C8
:1008200074206D656E7500557365206E756D62651B
:100830007273205B302D395D20746F20656469749C
:1008400020706172616D657465727300202D205394
:10085000797374656D20636F6E6669677572617414
:10086000696F6E000A0A6F70656E4C52536E672096
:10087000005129204F7574707574206265666F721F
:1008800065206C696E6B20283D465329203A200074
:10089000502920536C617665206D6F646520286552
:1008A00078706572696D656E74616C293A20004FCD
:1008B000292054696D65642042494E4420617420AA
:1008C0007374617274757020203A20004E29205094
:1008D000504D206F7574707574206C696D69746506
:1008E0006420202020203A200044495341424C45B6
:1008F00044004D292050504D205253534920746FCD
:10090000206368616E6E656C202020203A20004CC8
:10091000292050504D206D696E696D756D20737979
:100920006E63202875732920203A200044495341E2
:10093000424C4544004B29204661696C73616665F1
:1009400020626561636F6E20696E74762E20283197
:100950002D32353573293A20004A29204661696CC9
:100960007361666520626561636F6E2064656C61AA
:10097000792028302D323535203D3E20313073200E
:100980002D203135306D696E293A200049292046E5
:1009900061696C7361666520626561636F6E206674
:1009A00072712E203A200048292050574D20737430
:1009B0006F702064656C6179202020202020203A0F
:1009C000200047292050504D2073746F70206465BB
:1009D0006C6179202020202020203A200046292008
:1009E0004661696C736166652064656C617920207D
:1009F00020202020203A200050574D206368616E4F
:100A00006E656C200066756E6374696F6E3A2000C7
:100A10002920706F72742000506F776572546F7761
:100A2000657200445446205548462033322D626991
:100A3000742031306368004F70656E4C52536E679E
:100A40005258206D696E6920342F36636800466CF9
:100A50007974726F6E2F4F72616E676552582055B0
:100A600048462038636800525820747970653A20EF
:100A70000044697361626C656400487A00203D3D02
:100A8000200043616C63756C617465642070616300
:100A90006B657420696E74657276616C3A200042F1
:100AA00029204D6963726F202868616C6629205087
:100AB000504D202020203A00412920496E76657251
:100AC0007465642050504D20696E20202020203A0B
:100AD000003029204D7574652062757A7A65722020
:100AE000286D6F73746C79293A0039292053657227
:100AF00069616C2062617564726174653A00736D3E
:100B0000617274506F7274004672536B7900547244
:100B1000616E73706172656E740044697361626CBA
:100B200065640038292054656C656D657472793A86
:100B300020202020202020003729204368616E6E6D
:100B4000656C20636F6E6669673A20200036292045
:100B500044617461726174652028302D32293A2015
:100B6000202000352920486F70206368616E6E6513
:100B70006C733A2020202020003429204368616EC5
:100B80006E656C2073706163696E673A2020003374
:100B90002920524620706F7765722028302D372922
:100BA0003A202020003229205246206D6167696377
:100BB0003A202020202020202020003129204261BE
:100BC0007365206672657175656E63793A202020C1
:100BD0000000000000240027002A0000000000257B
:100BE0000028002B0000000000230026002900043C
:100BF00004040404040404020202020202030303C4
:100C000003030301020408102040800102040810BD
:100C1000200102040810200000000700020100006B
:100C20000304060000000000000000006D2E1124E7
:100C30001FBECFEFD8E0DEBFCDBF13E0A0E0B1E034
:100C4000ECE1FFE502C005900D92A639B107D9F796
:100C500016E0A6E9B3E001C01D92A934B107E1F79F
:100C60001CE0CEE2DCE004C02297FE010E94692F66
:100C7000CC32D107C9F70E94B22E0C948C2F0C9461
:100C80000000A0E0B0E0E7E4F6E00C94382FEC01BF
:100C9000A880B980CA80DB80A114B104C104D1044A
:100CA00041F484E2A82E89EDB82E8BE5C82E87E0AA
:100CB000D82EC601B5012DE133EF41E050E00E948E
:100CC000152F27EA31E440E050E00E94C12E7B015D
:100CD0008C01C601B5012DE133EF41E050E00E94E7
:100CE000152FCA01B9012CEE34EF4FEF5FEF0E94D0
:100CF000C12E6E0D7F1D801F911F97FF04C0615094
:100D0000704080409048688379838A839B839B01ED
:100D1000AC015F77B901CA01CDB7DEB7EAE00C9448
:100D2000542F0E944106089581EB92E00E944106F3
:100D300008956093B1027093B2028093B3029093CE
:100D4000B4020895A0E0B0E0E8EAF6E00C94312F98
:100D5000EC012B016A016115710519F0FB0191830A
:100D60008083C114D10449F0C6010297839728F00B
:100D700020E030E040E050E0DCC0A9908A2D90E017
:100D80000E94812F892BC9F7FDE2AF1621F4A990AB
:100D90003324339405C08BE2A81609F4A9903324B8
:100DA000C114D10421F0E0E1CE16D10411F5F0E335
:100DB000AF1669F48881883711F0883541F4A9802D
:100DC000229682E0382A20E1C22ED12C12C0C11412
:100DD000D10479F4E0E3AE1659F199E9E92E99E9E5
:100DE000F92E99E9092F99E1192F8AE0C82ED12C03
:100DF0003AC0FAE0CF16D10491F080E1C816D104D0
:100E000029F0E8E0CE16D104F9F415C0BFEFEB2EBF
:100E1000BFEFFB2EBFEF0B2FBFE01B2F24C0A9E9B4
:100E2000EA2EA9E9FA2EA9E90A2FA9E11A2F1BC077
:100E3000F8E0CF2ED12CEFEFEE2EEFEFFE2EEFEFFE
:100E40000E2FEFE11E2F0FC09601442737FD40956E
:100E5000542F6FEF7FEF8FEF9FEF0E94F32EC901AA
:100E6000DA017C018D0120E030E040E050E060E0FC
:100E70003601882477FC8094982C70EDB72EBA0C3C
:100E8000F9E0FB1570F48A2D81548A3118F499EC3D
:100E9000B92E06C08A2D81568A3148F589EAB82EC6
:100EA000BA0C8B2D90E08C159D050CF56F3FE9F089
:100EB000E216F30604071507B8F0CA01B901A40148
:100EC00093010E94C12E9B01AC018B2D90E0A0E00C
:100ED000B0E0280F391F4A1F5B1F281739074A0740
:100EE0005B0710F061E001C06FEFA990C6CF41141D
:100EF000510451F0662311F0219703C031FE04C064
:100F00002297F201D183C08330FE07C050954095EF
:100F1000309521953F4F4F4F5F4F67FF0AC082E2E8
:100F200090E090934806809347062FEF3FEF4FEFF6
:100F30005FEFB901CA01CDB7DEB7E1E10C944D2FE7
:100F4000FC0188279927E89421912032E9F3293080
:100F500010F02E30C8F32B3241F02D3239F4689462
:100F600004C00E94F507820F911D219120532A3061
:100F7000C0F31EF4909581959F4F089546E953E084
:100F80000E94C3070895009731F4DA018D919C9176
:100F9000009709F40EC0DC01FB013D912191222351
:100FA00019F03217C9F3FACF332331F4DA011D9265
:100FB0001C928827992708951197AF93BF93FB013F
:100FC0003D912191321771F4332321F48827992719
:100FD000119702C01E921196FA01A193B0839F91BE
:100FE0008F910895222369F7EACF7AE0979F902D99
:100FF000879F802D910D1124089580919803813051
:1010000019F482E08093980380919803833019F457
:1010100084E0809398030895E3E0F0E089E0809312
:101020005700849190E08670863009F491E0892F12
:1010300008951F93182F0E940C08882379F09FB7FA
:1010400081E080938F05F894A89588E180936000F3
:1010500010936000112309F0A8959FBF1F91089578
:10106000382F20E080912105909122058227932737
:1010700040E061E270E19C01220F331F97FF04C042
:10108000C9018627972701C0C9014F5F483099F7EA
:101090009093220580932105089586E38093BE03F3
:1010A00080E092ECA1E0B0E08093BF039093C00396
:1010B000A093C103B093C20387E08093CB0380EC7D
:1010C00092E9ADEEB9E18093C3039093C403A0937A
:1010D000C503B093C60385E08093CC038DEE9EEFED
:1010E000ADEABEED8093C7039093C803A093C903F4
:1010F000B093CA03ADECB3E080E090E0863010F02E
:10110000E0E004C0FC01E058FC4FE081ED93019663
:101110008831910599F782E08093E5038AE0809316
:10112000E603089580EC91EDA8E9BBE180939B0371
:1011300090939C03A0939D03B0939E0310929F03F2
:101140001092A0031092A1031092A2030895843676
:10115000910520F4BC0180E090E025C08E3B910514
:1011600050F48A559040BC0180E090E02AE030E0E5
:1011700040E050E016C0823D910550F4845B904001
:10118000BC0180E090E024E630E040E050E009C09F
:101190008D5C9040BC0180E090E028E532E040E0CA
:1011A00050E00E94C12E24E630E040E050E00E9472
:1011B000C12E089590E08C599F4F0E94A708089572
:1011C000DC019896EC91F0E0E770F070E858FC4F85
:1011D000808108958F929F92AF92BF92CF92DF92BB
:1011E000EF92FF920F931F938C010E94E008D801A9
:1011F00097962C9130E043E150E0249FF001259F29
:10120000F00D349FF00D1124EB54FD4F8080918040
:10121000A280B38090E00F96AA2797FDA095BA2FE1
:10122000BC01CD0120E43FE14DE750E00E94C12E1A
:10123000A50194010E94F32E69017A0180ED97E0E7
:10124000A0E0B0E0C80ED91EEA1EFB1ED801989699
:101250008C91887181F060E07EEE8AEB9BE0A501C5
:1012600094010E94F32E28513C4F4F4F5F4FC20E06
:10127000D31EE41EF51E87EE93E0A0E0B0E0C80E9A
:10128000D91EEA1EFB1EC701B60128EE33E040E07E
:1012900050E00E94F32ECA01B90128EE33E040E08D
:1012A00050E00E94C12E1F910F91FF90EF90DF90B0
:1012B000CF90BF90AF909F908F9008958F3F9105F2
:1012C00009F010F480E0089522E08030920710F4D5
:1012D00081E008958050934010F083E0089582E00B
:1012E0000895CF92DF92FF920F931F93CF93DF93D6
:1012F000F82FEB016A01182F1695E0E0888199819B
:10130000D6018C938A819B8111968C9311978C8145
:101310009D8112968C9312978E819F8113968C9348
:101320001397288139814A815B816C817D818E810F
:101330009F819295990F990F907C832F8370982BA2
:10134000852F8370880F880F982B872F8370829545
:10135000807F982B14969C9385E090E0C80ED91E50
:101360002896EF5F1E1750F6F0FF21C08881998103
:101370000E945E09F82E8A819B810E945E09182FC7
:101380008C819D810E945E09082F8E819F810E9421
:101390005E09F294FF0CFF0C70ECF7221295107F9F
:1013A0001F29182B000F000F012BD6010C93DF9182
:1013B000CF911F910F91FF90DF90CF90089523E080
:1013C0008032920718F420E030E026C023E0883E07
:1013D000920748F49C012F51334054E036952795ED
:1013E0005A95E1F719C027E0803D920720F49C014F
:1013F0002C5D334011C028E08839920718F02FEF98
:1014000033E00AC09C01285C374044E036952795BC
:101410004A95E1F72D503C4FC90108958C30910554
:1014200048F49C0174E0220F331F7A95E1F7285DA0
:101430003C4F17C023E0843F920720F49C012452C4
:101440003C4F0FC024E08030920718F020E938E0CC
:1014500008C09C012657334F64E0220F331F6A9562
:10146000E1F7C90108959C013695279525753575D5
:10147000821B930B9C0136952795369527952373F0
:10148000337383739373280F391FC901E4E0969572
:101490008795EA95E1F7820F931F8F709F7021E087
:1014A00031E0AC01429FC001439F900D529F900DCF
:1014B0001124892F0895882339F02D9800002B9A44
:1014C00000002D9A000008952D9800002B98000030
:1014D0002D9A000008952D9A000083B12D980000E8
:1014E00090E0B4E096958795BA95E1F781700895FC
:1014F0000F931F93082F5C9A2D985C9810E0802F13
:1015000080780E945B0A000F1F5F1830C1F72D988A
:101510001F910F9108958F770E94780A08950F9375
:101520001F93082F10E0802F80780E945B0A000F25
:101530001F5F1830C1F72D981F910F9108950F93D9
:101540001F932D9880E000E0182F110F0E946B0A66
:10155000810F0F5F0830C1F71F910F9108950E940E
:101560008B0A0E949F0A5C9A08951F93162F806829
:101570000E94780A812F0E948F0A5C9A1F91089519
:101580001F931091C7031827EEEBF3E0E80FF11D4E
:1015900089E767850E94B50A8DE3612F0E94B50A2D
:1015A00082E4612F0E94B50A1F91089586E20E948D
:1015B000AF0A08950F931F938C018CE1F8016481A9
:1015C0000E94B50A8DE1F80165810E94B50A8EE19D
:1015D000F80166810E94B50A80E2F80167810E94E5
:1015E000B50A81E2F80160850E94B50A82E2F8013D
:1015F00061850E94B50A83E2F80162850E94B50AFE
:1016000084E2F80163850E94B50A85E2F8016485E9
:101610000E94B50A8AE2F80165850E94B50A8EE645
:10162000F80166850E94B50A8FE6F80167850E9479
:10163000B50A80E7F80160890E94B50A81E7F801E0
:1016400061890E94B50A82E7F80162890E94B50AA1
:101650001F910F910895EF92FF920F931F93CF93D5
:10166000DF937B018C01603028E372072CE982074D
:101670002CE1920728F520E836E948E950E00E947D
:10168000F32EE9016897B90180E090E020E839E69F
:1016900047E65FEF0E94C12E6E0D7F1D801F911FD8
:1016A00032E0660F771F881F991F3A95D1F721E71F
:1016B00032E040E050E00E94F32E890180E421C036
:1016C00020E03DE241E351E00E94F32EE9016897FA
:1016D000B90180E090E020E033ED4EEC5EEF0E9437
:1016E000C12E6E0D7F1D801F911F660F771F881FF3
:1016F000991F21E732E040E050E00E94F32E89017B
:1017000080E69E012F71622F680F85E70E94B50A5F
:1017100086E7612F0E94B50A87E7602F0E94B50A0D
:10172000CDB7DEB7E6E00C94582F9F92AF92BF92F0
:10173000CF92DF920F93DF93CF9300D000D0CDB73D
:10174000DEB7982E83E00E94AF0A8093E70384E01F
:101750000E94AF0A8093E80386E060E00E94B50A29
:1017600087E061E00E94B50A89E06FE70E94B50A50
:101770008AE065E00E94B50A8BE062E10E94B50A4A
:101780008CE065E10E94B50A8DE06DEF0E94B50A1C
:101790008EE060E00E94B50A992019F084E193E0A0
:1017A00008C08091E50323E1829FC00111248B547E
:1017B0009D4F0E94DA0A80E36CE80E94B50A82E33A
:1017C0006FE00E94B50A83E362E40E94B50A84E3F5
:1017D0006AE00E94B50A85E36AE20E94B50A86E3E0
:1017E0006DE20E94B50A87E364ED0E94B50A88E3C2
:1017F00060E00E94B50A89E360E00E94B50A992082
:1018000049F065E7A62E61ECB62E61ECC62E6EEDB2
:10181000D62E08C0A090C703B090C803C090C903DB
:10182000D090CA030AE38D2D9927AA27BB27898365
:101830009A83AB83BC83802F69810E94B50A802F75
:101840008B5F69810E94B50ADC2CCB2CBA2CAA24B0
:101850000F5F0E3341F783E46FEF0E94B50A84E413
:101860006FEF0E94B50A85E46FEF0E94B50A86E427
:101870006FEF0E94B50A992019F08DE666E003C06B
:101880008DE66091CB030E94B50A89E760E00E9473
:10189000B50A8AE76091CC030E94B50A83E760E04D
:1018A0000E94B50A84E760E00E94B50A992029F0F9
:1018B00060EC72E98DEE99E108C06091C30370910C
:1018C000C4038091C5039091C6030E942B0B0F9017
:1018D0000F900F900F90CF91DF910F91DF90CF90ED
:1018E000BF90AF909F90089587E061E00E94B50A95
:1018F0008EE764E20E94B50A88E063E00E94B50AC0
:1019000088E060E00E94B50A87E065E00E94B50AC1
:1019100085E062E00E94B50A83E00E94AF0A8093EE
:10192000E70384E00E94AF0A8093E8030895582FEC
:1019300040918C04842F90E0FC01EF70F0709F01C7
:101940002F5F3F4F74E0959587957A95E1F72817BB
:10195000390751F0E458FB4F5083842F8F5F8F700D
:10196000407F842B80938C0408951F920F920FB6B2
:101970000F9211241F932F933F934F935F936F9375
:101980007F938F939F93AF93BF93CF93DF93EF9307
:10199000FF93C0918600D09187002091CE043091B2
:1019A000CF048091AD04882309F047C0CE01821B8B
:1019B000930B9C0180919F0385FD02C0369527956E
:1019C00099E0253C390708F1809147038630D0F033
:1019D000809147038F3FB1F020E00EC0E22FF0E08E
:1019E000EE0FFF1FDF01A255BB4F8D919C91E95D6A
:1019F000FC4F918380832F5F80914703281770F3FA
:101A00001092AC041092470318C082E02D3B3807B7
:101A100060F180914703803140F510914703C9017F
:101A20000E94DF09E12FF0E0EE0FFF1FE255FB4FB0
:101A3000918380831F5F10934703D093CF04C0939B
:101A4000CE04FF91EF91DF91CF91BF91AF919F9124
:101A50008F917F916F915F914F913F912F911F9146
:101A60000F900FBE0F901F9018958FEF8093470334
:101A7000E4CF83E0809380008AE9809381008091A5
:101A80009F0386FD05C08091810080648093810062
:101A90008FEF9FEF909389008093880080916F0073
:101AA000806280936F0008956F3020F08695869550
:101AB000805408958DE0689F802D11240895882317
:101AC00019F460E071E002C063E071E085E296E045
:101AD0000E94752C0895A0E0B0E0E1E7FDE00C94D1
:101AE0003A2F182F0E9448299B01AC0180911B05B9
:101AF00090911C05A0911D05B0911E0569017A0108
:101B0000C81AD90AEA0AFB0AD701C60189589341C3
:101B1000A040B04010F010921A0520931B0530939E
:101B20001C0540931D0550931E052091AD04822F86
:101B300081508230E8F580911A05882309F44FC15D
:101B4000813011F482E0BCC1803108F035C1E82F4A
:101B5000F0E0E255FB4F10838F5F80931A058031D0
:101B600009F0B0C1A0EBB4E0213039F41196EC914A
:101B70001197E695E6958C9109C08D919C911197EE
:101B8000E92FE695E695E69596958795E03140F440
:101B9000F0E090E0EE0FFF1FE95DFC4F9183808342
:101BA0001092AC04129684E0AE3BB807E9F68AC105
:101BB000233009F004C180911A05882321F41F30D5
:101BC00009F080C10CC1883130F4E82FF0E0E35512
:101BD000FB4F108374C1883109F0EEC0112309F066
:101BE000EBC0C0E0D0E00BE010E0DE0163E0AA0F44
:101BF000BB1F6A95E1F7C09FB001C19F700DD09FD8
:101C0000700D1124FB01E255FB4F80812181922F41
:101C1000977095958795FD01EE0FFF1FE95DFC4FCD
:101C200091838083FB01E155FB4F308136953695DA
:101C300036952181422F4295440F407E842F832B7D
:101C4000269526952695922F977095958795FD0157
:101C5000EE0FFF1FE75DFC4F91838083FB01E05592
:101C6000FB4F808182958695869583704181942F64
:101C7000990F990F292F282B429546954695437029
:101C800082818170880F880F382F342B35952795E6
:101C9000FD01EE0FFF1FE55DFC4F31832083FB014B
:101CA000EE54FB4F308136952181422F47954427D2
:101CB0004795842F832B2695922F9770959587951E
:101CC000FD01EE0FFF1FE35DFC4F91838083FB015D
:101CD000ED54FB4F308132953F702181422F429568
:101CE000407F842F832B22952F70922F977095958C
:101CF0008795FD01EE0FFF1FE15DFC4F918380830F
:101D0000FB01EC54FB4F8081881F8827881F41818D
:101D1000942F990F292F282B441F4427441F828179
:101D20008370880F382F342B35952795FD01EE0FE2
:101D3000FF1FEF5CFC4F31832083FB01EA54FB4F14
:101D40003081369536952181422F4295440F440FBC
:101D5000407C842F832B26952695922F97709595FE
:101D60008795AA0FBB1FFD01ED5CFC4F918380831B
:101D700069547B4FFB012081229526952770418174
:101D8000342F330F330F330F832F822B942F9295E1
:101D90009695977095958795AB5CBC4F11969C93E3
:101DA0008E932196C230D10509F01FCF8091C404D3
:101DB00083FD02C01092AC0410921A0583C0243037
:101DC00009F080C040911A05442359F4183AB1F43F
:101DD000109222051092210588EA0E94300881E0C5
:101DE0006FC0413019F410931F0504C0423031F424
:101DF00010932005812F0E9430085DC0609120055E
:101E0000262F30E0220F331FE42FF0E0C9010296A5
:101E10008E179F0734F0433268F7E555FB4F108368
:101E2000E9CF2D5F3F4F4091210550912205E217E8
:101E3000F30749F4912F80E0482759275093220552
:101E40004093210538C0812F90E04817590789F544
:101E500080911F05813069F5613118F080E1809330
:101E60002005D09020054EEAE42E44E0F42E00E058
:101E700010E01BC0F701D081C0E0818190E08C2B85
:101E80009D2B33E0969587953A95E1F70E94DF09FF
:101E9000F801EE0FFF1FE95DFC4F918380830F5F18
:101EA0001F4F82E090E0E80EF91E0D1518F3109216
:101EB000AC0410921A0580911A05882319F08F5FDF
:101EC00080931A05CDB7DEB7E8E00C94562FFF9249
:101ED0000F931F93CF93DF93182F092FF62E8EE3C6
:101EE0000E94B50A212F302FC901EC0110E005C076
:101EF0008FE769910E94B50A1F5F1F15C8F385E03F
:101F000064E00E94B50A83E00E94AF0A8093E70371
:101F100084E00E94AF0A8093E8030E9448296093FE
:101F2000E9037093EA038093EB039093EC0387E05B
:101F300069E00E94B50A81E080939803CDB7DEB7CF
:101F4000E5E00C94592F0E94670F8091980381302F
:101F5000D9F40E9448292091E9033091EA03409185
:101F6000EB035091EC03621B730B840B950B605ACF
:101F700076488140904040F4E8CF85E296E067E003
:101F800071E00E94752C0895809198038130A9F327
:101F9000089585E296E06EE70E942D2E0895A0E058
:101FA000B0E0E5EDFFE00C94392F6C0185E296E09E
:101FB0006EE70E942D2E760100E010E0C0E0D0E038
:101FC000B0E2BB2E0AC00830110521F49E01209515
:101FD000F60120870894E11CF11CF7016081862F2F
:101FE0008D57823040F485E296E06DE70E942D2EF9
:101FF000F70160816B2585E296E00E942D2E011588
:10200000110551F0F70180819E01280F311DC32F6A
:10201000DD27C20FD31FD0700F5F1F4F093011058E
:1020200091F6CDB7DEB7E9E00C94552FA9E0B0E00A
:10203000ECE1F0E10C94402F382FE62F80919104D1
:1020400090E0019664E270E00E94E02E982F809369
:10205000910488E9898380E18A83913071F091301D
:1020600028F0923099F09330E1F416C085E08B832C
:1020700081EF8C832F5F2D8317C09B8381EF8C832F
:1020800084E6489FC00111249D830EC084E08B83A9
:1020900081EF8C833D8308C09B8381EF8C83ED832C
:1020A00003C00E94C90F04C0CE0101960E94CF0F49
:1020B0002996E2E00C945C2F0F931F93CF93DF934C
:1020C000182F092F85E296E06EE70E942D2E212F12
:1020D000302FC901EC0110E000E288818D57823079
:1020E00040F485E296E06DE70E942D2E88818027DE
:1020F000888385E296E069910E942D2E1F5F19303A
:1021000061F785E296E06EE70E942D2EDF91CF9178
:102110001F910F910895A9E0B0E0E1E9F0E10C947E
:10212000402F382F80919104882379F48EEF898392
:102130003A836B83842F90E0959587958C832D83CC
:10214000198618861F821E822FC040918C04842F0E
:1021500090E09C012F70307054E0959587955A95CA
:10216000E1F78217930721F18DEF89831A821B8291
:10217000DE01149620E008C0E458FB4F80818D9367
:10218000405F2F5F263069F0842F90E0FC0134E03F
:10219000F595E7953A95E1F78F709070E817F90794
:1021A00059F740938C042A83CE0101960E945C105B
:1021B0008091910490E0019666E070E00E94E02E2C
:1021C000809391042996E2E00C945C2F9F92AF9249
:1021D000BF92CF92DF92EF92FF920F931F93B82E90
:1021E000A62ED42EC22E902E0E9448297B018C014F
:1021F00080917B0420918D0430918E0440918F0456
:10220000509190048823B1F0D801C701821B930B31
:10221000A40BB50B815E9E42A040B04020F12C2D56
:10222000DC1408F42D2D8B2D6A2D422F292D0E94B0
:10223000161011C0D801C701821B930BA40BB50B5C
:1022400081539547A040B04070F08B2D6A2D4D2DE5
:102250002C2D0E948B10E0928D04F0928E0400933E
:102260008F04109390041F910F91FF90EF90DF90D7
:10227000CF90BF90AF909F90089585E296E06091D7
:10228000EE030E942D2E08951F93182F85E296E0ED
:10229000612F0E942D2E8091EE0381278093EE0303
:1022A0001F9108951F93192F0E944411812F0E949E
:1022B00044111F910895DF92EF92FF920F931F93A5
:1022C000D82E7B011092EE0305E216E0C80165EB03
:1022D0000E942D2EC80162E60E942D2E8D2D0E9497
:1022E0004411C7010E9452111F910F91FF90EF906E
:1022F000DF9008958CE060E00E94CD298BE061E0E2
:102300000E94CD298DE061E00E94CD2982E060E04D
:102310000E94CD2984E061E00E94CD290895892B97
:1023200019F08FE061E002C08FE060E00E94392A7E
:102330000895A0E0B0E0EFE9F1E10C94382F8CE0D3
:102340000E94AF0A882389F585E296E063E171E097
:102350000E94752C5E9A409A80E00E94950B0E9424
:10236000740C5E98409821C085E296E00E94F42D9E
:10237000482F8091AD04882321F0842F0E946B0D9B
:1023800014C080911805E82FF0E031969F012F715D
:10239000307031978091170590E02817390729F0A0
:1023A000E251FB4F40832093180585E296E00E949E
:1023B000BA2D892BC9F680919803843009F08CC01E
:1023C0000E94482960939C0470939D0480939E040E
:1023D00090939F04611571058105910561F481E079
:1023E00090E0A0E0B0E080939C0490939D04A093C3
:1023F0009E04B0939F048091A8049091A9048160E9
:102400009093A9048093A80483E0809398038FE7B6
:102410000E948B0AC5EED4E00E949F0A899304E0D3
:10242000CE3ED007C9F74091D0048091E504282F13
:1024300030E0842F90E08227932786FF40C080E41D
:1024400048274093D004C90188739070C89709F554
:1024500010E014C01F5F8091E603E12FF0E084FFDD
:1024600006C0EB51FB4F80810E94970C07C0EB51D7
:10247000FB4F85E296E060810E942D2E212F30E0F7
:102480008091E50490E0877090708217930714F7AD
:1024900016C02F733070232B91F48091E604809343
:1024A000A0048091E7048093A2048091E8048093C3
:1024B000A3048091EB048093AA041092AB04809152
:1024C0001905813019F482E080931905809119056E
:1024D000833011F4109219050E9448295B016C01A8
:1024E0008091A4049091A504A091A604B091A704A2
:1024F0000097A105B105C9F0A6019501281B390B6C
:102500004A0B5B0BDA01C901885B9B40A040B040DD
:1025100060F00E94D60A8093A1041092A404109245
:10252000A5041092A6041092A7048EEB93E00E94DB
:10253000EA08209198043091990440919A045091AE
:102540009B0486017501E21AF30A040B150BE616CB
:10255000F7060807190708F4EEC0A0929804B09295
:102560009904C0929A04D0929B04A8958091AC04DF
:10257000883008F0D7C08091AC048F5F8093AC04A2
:10258000E0909C04F0909D0400919E0410919F04A3
:10259000E114F1040105110511F18EEB93E00E94A5
:1025A000EA08AE18BF08C00AD10A6A157B058C0577
:1025B0009D0588F480919F0384FD04C080ED97E021
:1025C0000E948F1110929C0410929D0410929E0400
:1025D00010929F0404C080E090E00E948F119091BF
:1025E000D004907C9093D0040091180510911705A9
:1025F0000117B1F180911905823091F590589093AF
:10260000D0048EEB93E00E94E008893010F048E09F
:1026100002C0482F415030E013C03F5FA32FB0E00D
:10262000812F90E0FC01E251FB4F2081FD01E0533E
:10263000FB4F2083A25FBA4F2C930196182F1F7176
:10264000341710F4101749F710931705832F895C7E
:102650009091D004892B8093D00430930E051AC03A
:10266000209119052430D1F490910E05EFE0F5E0AA
:10267000A1EDB4E0292F30E02E0F3F1F02C0819161
:102680008D93E217F307D9F7995C8091D004982BCA
:102690009093D00483E08093190525C08091930422
:1026A000823031F491609093D0045E9A409A10C0C9
:1026B0009093D0045E984098222319F481E080938F
:1026C000190580911905833019F484E08093190568
:1026D000F8948091E603877067E273E041ED54E07F
:1026E0000E94710978945D9A419A809192040E94A7
:1026F000C00A8EEB93E00E94E008682F80ED94E022
:102700000E94670FE0919204EF5FE0939204E8313A
:1027100031F0F0E0E254FC4F8785882361F4109299
:10272000920409C08091AC04883011F45E9A409AFA
:1027300089E08093AC048091E603887171F1809107
:102740009803823051F58091A8049091A904880FD4
:10275000991F9093A9048093A80483E08093980321
:102760000E94740C0E9448296093A4047093A504ED
:102770008093A6049093A7046115710581059105C6
:1027800061F481E090E0A0E0B0E08093A404909335
:10279000A504A093A604B093A7048091E60384FF48
:1027A0001EC08091A8049091A9048E7F0E94330AD4
:1027B000182F8091A0046091AA040E94540D082F44
:1027C0008091A104612F0E94540D282F8091A204B2
:1027D0006091A304402F009199030E94E6105D9838
:1027E0004198809193048130C9F0813020F082308B
:1027F00009F03FC033C083E10E946C2A892BC9F5E0
:1028000081E0809393040E943A296093940470932A
:10281000950480939604909397042BC083E10E94C3
:102820006C2A892B21F50E943A2920919404309139
:1028300095044091960450919704621B730B840B8E
:10284000950B695E73408040904098F082E08093E1
:10285000930480ED97E00E948F110BC083E10E94EA
:102860006C2A892B31F080E090E00E948F11109249
:102870009304CDB7DEB7EAE00C94542F8FE061E00B
:102880000E94CD298FE060E00E94392A08951F93AD
:10289000182F0E94482960938D0470938E048093B2
:1028A0008F049093900410937B04112329F440E843
:1028B00055E260E070E004C040E051EE60E070E09E
:1028C00085E296E00E94332D1F910895ACE1B0E0BF
:1028D000ECE6F4E10C94382F0E9448297B018C012E
:1028E00081E00E94950BA4E7AA2E6E010894C11CFA
:1028F000D11CF3E0BF2EA982C60161E00E94A30FA4
:10290000B09298030E94740C6AEF70E080E090E04F
:102910000E946E2980919803833009F07DC085E282
:1029200096E00E94BA2D892B09F076C00E944829B2
:102930006E197F09800B910B6058734C894C914044
:1029400008F06AC0D8CF8FE70E948B0A0E949F0AC6
:10295000843509F05CC089830E949F0A182F00E02B
:1029600010937A04009379040E949F0A080F111DA6
:1029700010937A04009379040E949F0A809378044C
:102980000E949F0A80937704813108F040C0FF24A1
:1029900007C00E949F0A095A1B4FF8018083F394D5
:1029A0000F2D10E08091770490E0880F991F081791
:1029B000190778F380E78983CE01019661E00E94D0
:1029C000A30F83E0809398030E94740C62E370E08D
:1029D00080E090E00E946E29809198038330A9F0F6
:1029E0008FE70E948B0A0E949F0A803581F48983B9
:1029F00003EA13E00E949F0AF80181938F01F3E03C
:102A00000E3B1F07B9F781E003C082E001C083E0FD
:102A10006C96EAE00C94542F80919803833009F06F
:102A200092CFF3CF83E00E94AF0A8093E70384E064
:102A30000E94AF0A8093E80387E061E00E94B50A34
:102A40006AE070E080E090E00E946E290E94740CC1
:102A5000000008950F931F93082F19C05E9A409AA3
:102A600064E670E080E090E00E946E295E984098F5
:102A700064E670E080E090E00E946E291F5F10170E
:102A800068F36CE271E080E090E00E946E2910E053
:102A9000F6CF482F392F25E00DC0F999FECF1FBA88
:102AA000842F932F92BD81BD60BD0FB6F894FA9A22
:102AB000F99A0FBE215059F0F999FECF842F932F28
:102AC00092BD81BDF89A80B5681739F7089582E004
:102AD0000E942A150895A0E0B0E0E1E7F5E10C942A
:102AE000312F482E562EEE24FF2488249924C0E04E
:102AF000D0E0CC24DD2436E3332E04C0CC24DD2406
:102B000055245394442069F480919903839DE001F6
:102B100011242AE9E22E23E0F22E99E0892E912C4D
:102B20001DC021E0421671F480919903839DE0015C
:102B300011242B968EEBE82E83E0F82E09E2802EEE
:102B4000912C0CC032E0431649F419E9E12E13E050
:102B5000F12EB1E08B2E912CC8EDD0E03E016C0C33
:102B60007D1C1092220510922105E3011BC0552007
:102B700059F4F999FECFD2BDC1BDF89A80B5F701DD
:102B8000E00FF11F808307C0F701E00FF11FCE01B6
:102B900060810E9449150E0D1F1DF80180810E9461
:102BA000300821969E012619022F10E008151905FC
:102BB000F0F2CE015520D9F4F999FECFD2BDC1BDB6
:102BC000F89A20B5F999FECF2196D2BDC1BD2197C3
:102BD000F89A80B590E0B22EAA248A299B292091E8
:102BE0002105309122052817390759F487CF2196FE
:102BF000609122050E944915CE01609121050E9435
:102C0000491580E091E0C80ED91E91E0C91693E005
:102C1000D90608F477CF852DCDB7DEB7E1E10C9466
:102C20004D2F80E061E00E946B1581E061E00E9421
:102C30006B15089580E060E00E946B15882331F0E9
:102C400081E060E00E946B15882331F40E949208B5
:102C50000E944D080E941116089582E061E00E94D2
:102C60006B15089582E060E00E946B1580919903D6
:102C7000843020F0109299030E942D1608951F931E
:102C8000182F0E94321680919903811731F0143069
:102C900020F4109399030E942D161F91089510920D
:102CA000550485E6E0EFF3E0DF011D928A95E9F730
:102CB00008951F93182F8F3711F08830E1F5E091B8
:102CC0005504EE2309F455C0E150E0935504F0E0BB
:102CD000E051FC4F108285E296E06DE00E942D2EBF
:102CE00010E00AC0E12FF0E0E051FC4F85E296E0F1
:102CF00060810E942D2E1F5F80915504181790F35C
:102D000085E296E060E20E942D2E85E296E06DE07D
:102D10000E942D2E10E00AC0E12FF0E0E051FC4FA0
:102D200085E296E060810E942D2E1F5F8091550400
:102D3000181790F31CC08B3119F40E944F161FC056
:102D40008D30E9F08A30D9F080915504843688F4CA
:102D500085E296E0612F0E942D2E80915504E82F88
:102D6000F0E0E051FC4F10838F5F8093550480E0CA
:102D700007C085E296E067E00E94E12AF8CF81E093
:102D80001F9108951F93CF93DF93CDECD3E010E014
:102D90003BC085E296E062E271E00E94722C85E21F
:102DA00096E0612F4AE050E00E94EF2B85E296E02A
:102DB0006FE271E00E94722C699170E080E090E017
:102DC0002091CC0330E040E050E00E94C12E20E191
:102DD00037E240E050E00E94C12EDC01CB0140917F
:102DE000C3035091C4036091C5037091C603480F9B
:102DF000591F6A1F7B1F85E296E02AE030E00E949F
:102E0000B62B1F5F183119F08881882311F6DF91E6
:102E1000CF911F910895EF92FF920F931F938823F4
:102E200039F485E296E061E77AE00E94FF2A3BC030
:102E300090E00E94A70824E630E040E050E00E94C5
:102E4000F32E122F032FF42EE52E622F732F842FD3
:102E5000952F2AE030E040E050E00E94F32E85E21A
:102E600096E0BA01A9012AE030E00E94A72B85E292
:102E700096E06EE20E94E12A612F702F8F2D9E2D29
:102E80002AE030E040E050E00E94F32EAB01BC01AC
:102E900085E296E02AE030E00E94A72B85E296E0EA
:102EA00063E70E94132B1F910F91FF90EF900895FD
:102EB000FF920F931F93CF93DF9385E296E067E62F
:102EC0007AE00E94C02A8091A303813041F485E218
:102ED00096E06EE47AE00E94FF2AFF246DC0823003
:102EE00029F485E296E067E37AE0F5CF843029F4AF
:102EF00085E296E063E27AE0EECF853071F785E215
:102F000096E068E17AE0E7CFCF2DD0E0C930D10577
:102F10001CF06F2D685C02C06F2D6F5C85E296E03F
:102F20000E94E12A85E296E060E17AE00E94C02AF0
:102F3000BE016F5F7F4F85E296E04AE050E00E945D
:102F40004B2C85E296E065E07AE00E94C02A8E0173
:102F50000D551C4FD8011196EC91E032F8F485E242
:102F600096E068EF79E00E94C02AF8018181803103
:102F700030F085E296E063E371E00E94722CCD555B
:102F8000DC4F698170E06F7070706F5F7F4F85E21A
:102F900096E04AE050E00E945E2C0DC0F0E0EF7039
:102FA000F070EE0FFF1FE85BFC4F6081718185E2DE
:102FB00096E00E94752CF39480917804F81608F43A
:102FC000A3CF85E296E06DED79E00E94C02A809162
:102FD000BB030E940B1785E296E062EC79E00E9449
:102FE000C02A8091BC030E940B1785E296E067EA35
:102FF00079E00E94C02A8091BD030E940B1785E2F0
:1030000096E06CE879E00E94C02A4091B3035091A9
:10301000B4036091B5037091B60341155105610584
:10302000710539F185E296E02AE030E00E94B62B86
:1030300085E296E069E579E00E94C02A8091B703B5
:103040000E94DA08AB01BC0185E296E02AE030E09C
:103050000E94B62B85E296E065E379E00E94C02AE3
:1030600085E296E06091B8034AE050E00E94012CAE
:1030700006C085E296E06CE279E00E94FF2A85E2D4
:1030800096E06FE079E00E94C02A6091B9037091E8
:10309000BA0385E296E04AE050E00E94DB2B85E22D
:1030A00096E062EF78E00E94C02A6091B20360313E
:1030B00050F470E06F5F7F4F85E296E04AE050E0A9
:1030C0000E945E2C06C085E296E069EE78E00E94E0
:1030D000FF2A85E296E06CEC78E00E94C02A80919D
:1030E000B10380FD03C065E371E002C069E371E0F4
:1030F00085E296E00E94752C85E296E06FEA78E022
:103100000E94C02A8091B10382700E945F0D85E207
:1031100096E060E978E00E94C02A8091B103847053
:103120000E945F0D85E296E061E778E00E94C02A88
:103130008091B10388700E945F0DCDB7DEB7E5E0E6
:103140000C94592F1F93CF93DF9385E296E06BEB9E
:103150007BE00E94C02A4091C3035091C403609158
:10316000C5037091C60385E296E02AE030E00E9434
:10317000B62B85E296E065EA7BE00E94C02A40918A
:10318000C7035091C8036091C9037091CA0385E2D7
:1031900096E020E130E00E94B62B85E296E06FE8F1
:1031A0007BE00E94C02A85E296E06091CB034AE072
:1031B00050E00E94012C85E296E069E77BE00E94E6
:1031C000C02A85E296E06091CC034AE050E00E947C
:1031D000012C85E296E063E67BE00E94C02ACDECFC
:1031E000D3E010E012C0112331F085E296E06DE3E8
:1031F00071E00E94722C85E296E069914AE050E00D
:103200000E94EF2B1F5F183119F08881882359F72E
:1032100085E296E00E94E92A85E296E06DE47BE093
:103220000E94C02A85E296E06091E5034AE050E002
:103230000E94012C85E296E068E37BE00E94C02AB0
:10324000E091E603F0E0E770F070EE0FFF1FE85941
:10325000FC4F6081718185E296E00E94752C85E2C9
:1032600096E063E27BE00E94C02A8091E60390E052
:10327000887190708830910589F0893091051CF42F
:10328000892B39F01BC08031910569F04897B1F462
:103290000FC085E296E06AE17BE00EC085E296E031
:1032A0006EE07BE009C085E296E068E07BE004C068
:1032B00085E296E06EEF7AE00E94FF2A85E296E0D2
:1032C0006AEE7AE00E94C02A4091BF035091C00389
:1032D0006091C1037091C20385E296E02AE030E07C
:1032E0000E94B62B85E296E061ED7AE00E94C02A4A
:1032F00080919F0380710E945F0D85E296E068EBEC
:103300007AE00E94C02A80919F0380740E945F0D22
:1033100085E296E06FE97AE00E94C02A80919F03DF
:1033200080720E945F0D85E296E062E87AE00E947A
:10333000C02A8EEB93E00E94EA08AB01BC0185E253
:1033400096E02AE030E00E94A72B85E296E06DE748
:103350007AE00E94C02A8EEB93E00E94EA089B016B
:10336000AC0160E472E48FE090E00E94F32E85E20D
:1033700096E0BA01A9012AE030E00E94A72B85E27D
:1033800096E06AE77AE00E94FF2ADF91CF911F91D1
:103390000895EF92FF920F931F937C0105E216E0D0
:1033A000C8016F2D70E04AE050E00E94CA2BC801AE
:1033B0006EE20E94E12AB701E4E076956795EA950E
:1033C000E1F76F707070C8014AE050E00E94CA2BAC
:1033D000C8016EE20E94E12A8FE0E822FF24C801C2
:1033E000B7014AE050E00E94CA2B1F910F91FF9055
:1033F000EF9008950F931F93CF93DF932091EF03E6
:103400002F3FA9F585E296E061EF75E00E94C02AA2
:1034100083E693E00E94C91985E296E060ED75E0CD
:103420000E94C02A8091790490917A040E94C9195F
:1034300085E296E06DE975E00E94FF2A85E296E05C
:103440006AE775E00E94FF2A85E296E062E675E091
:103450000E94FF2A85E296E06DE375E00E94FF2A54
:1034600085E296E00E94E92A0E94581769C0121668
:103470000CF066C0332727FD30958091780490E0EA
:10348000821793070CF45CC085E296E068E275E071
:103490000E94C02A6091EF03772767FD709585E24F
:1034A00096E04AE050E00E945E2C85E296E06DEFE7
:1034B00074E00E94C02A08E210E03AC0C12FD0E0B8
:1034C000CC0FDD1FC95ADB4F288130E08091EF031C
:1034D000992787FD909501972817390741F585E2CF
:1034E00096E06FE371E00E94722C85E296E0602F17
:1034F0004AE050E00E94EF2B85E296E063E471E041
:103500000E94722CE981F0E0EF70F070EE0FFF1F67
:10351000E85BFC4F6081718185E296E00E94722C2D
:1035200085E296E067E471E00E94722C0F5F1F5FF6
:1035300080917704181710F285E296E00E94E92A3C
:10354000DF91CF911F910F910895ACE1B0E0EBEACC
:10355000FAE10C943A2F282F8091EF038F3F09F066
:1035600042C1822F90E0FC013A97EF36F10508F056
:1035700033C1EC5CFF4F0C94672F85E296E069E461
:1035800071E0AEC085E296E069E471E00E94752CBE
:103590001CC185E296E065E571E00E94752C85E727
:1035A0008983DE011296E3EAF3E08BE101900D924C
:1035B0008150E1F7CE0101966CE10E94A30F0E94B9
:1035C000740C83E08093980368EC70E080E090E0F6
:1035D0000E946E2980919803843009F0FDC08FE726
:1035E0000E948B0A0E949F0A8983853509F0F4C0E6
:1035F00085E296E06FED74E00E94FF2A85E296E096
:1036000061EC74E00E94FF2A85E296E063EA74E0D0
:10361000ACC085E296E06DE671E00E94752C89E60B
:103620008983CE01019661E00E94A30F0E94740C71
:1036300083E08093980368EC70E080E090E00E9463
:103640006E2980919803843009F0C6C08FE70E94EC
:103650008B0A0E949F0A89838E010E5F1F4F2DE106
:10366000E22EF12CEC0EFD1E0E949F0AD8018D93D4
:103670008D01AE15BF05C1F7A3EAB3E0FE01329696
:103680008BE101900D928150E1F78981893409F035
:10369000A3C085E296E065E874E00E94FF2A85E217
:1036A00096E067E674E00E94FF2A85E296E069E40E
:1036B00074E05BC085E296E067E871E00E94752CDB
:1036C0008EEF8093EF0388C020522750922F9053A3
:1036D00080917804891738F485E296E066E971E014
:1036E0000E94752C79C09093EF036FC084E18093A2
:1036F000EF0385E296E062E174E037C085E18093F4
:10370000EF0385E296E06BED73E02FC086E18093D6
:10371000EF0385E296E064EA73E027C087E18093D7
:10372000EF0385E296E06AE573E01FC088E18093CD
:10373000EF0385E296E069E473E017C089E18093C6
:10374000EF0385E296E065E373E00FC08AE18093C2
:10375000EF0385E296E060E273E007C08BE18093BF
:10376000EF0385E296E068EF72E00E94FF2A34C022
:1037700085E296E06EED72E00E94FF2A8091B1032F
:1037800091E01DC085E296E068EC72E00E94FF2A9D
:103790008091B10392E013C085E296E063EB72E0A2
:1037A0000E94FF2A8091B10394E009C085E296E06F
:1037B00068E972E00E94FF2A8091B10398E08927AE
:1037C0008093B1038FEF8093EF030E94FA1904C036
:1037D00085E296E00E94F42D85E296E00E94BA2DE3
:1037E000892BB1F762C1822F0E945916882309F4F0
:1037F0005CC180915504882321F48FEF8093EF03FF
:103800004CC180EF93E060E070E040E050E00E9447
:10381000A2069B01AC016091EF03862F992787FDDB
:103820009095A92FB92FFC013197EB31F10508F0E4
:1038300024C1ED55FF4F0C94672FE62FFF27E7FDBE
:10384000F0958091780490E08E179F070CF415C1D5
:10385000DA01C9010197A109B1098097A105B10554
:1038600048F098E2F92E00E010E06F010894C108DA
:10387000D10825C0ED55FC4F822F81508083E5C0D3
:10388000612F70E0660F771F695A7B4FFB018081C3
:1038900090E08C159D0591F48F2D90E0A0E0B0E0B4
:1038A00082179307A407B50741F4F601ED55FC4FC5
:1038B000DB0111968C91818301E0F3941F5F80916D
:1038C00077041817E8F2BFC02F3F310541055105B5
:1038D00011F008F0D2C02093BB03B7C02F3F3105D1
:1038E0004105510511F008F0C8C02093BC03ADC0DC
:1038F0002F3F31054105510511F008F0BEC020935E
:10390000BD03A3C08091F0038062803719F581EF79
:1039100093E060E070E040E050E00E94A2069B016E
:10392000AC01DC01CB010197A109B1090897A10500
:10393000B10508F0B5C0CA01B90124ED30E340E09B
:1039400050E00E94C12E9B01AC012A5E3C4A4A46CF
:10395000554E24C0863611F581EF93E060E070E0AB
:1039600040E050E00E94A2069B01AC01DC01CB01CB
:103970000197A109B1090797A105B10508F090C009
:10398000CA01B90128EA31E640E050E00E94C12EA8
:103990009B01AC01245E3C434E46544E211531053B
:1039A0004105510561F0DA01C9018054914EAD49DC
:1039B000B8418158904FAA4FB24008F05EC02093A2
:1039C000B3033093B4034093B5035093B6033DC0A3
:1039D0002F3F31054105510511F008F04EC02093ED
:1039E000B70333C0DA01C9010197A109B1098F3FBB
:1039F0009105A105B10508F040C02093B80325C08A
:103A0000DA01C901845C9940A040B0408D549D41C9
:103A1000A040B04030F43093BA032093B90301E0E2
:103A200001C000E0211531054105510511F48FEF6A
:103A300007C0213131054105510528F4822F8150FD
:103A40008093B20302C00023C1F080915604882302
:103A5000D1F48091C7039091C803A091C903B0919C
:103A6000CA030196A11DB11D8093C7039093C8039B
:103A7000A093C903B093CA0306C085E296E068EA42
:103A800071E00E94752C0E944F168FEF8093EF0318
:103A900085E296E06AE00E94132B0E94FA1905C0A5
:103AA00021E030E040E050E07ECF6C96E8E00C94FE
:103AB000562F85E296E06CE472E00E94FF2A85E2D0
:103AC00096E064E372E00E94FF2A85E296E00E949D
:103AD000BA2D892B31F085E296E00E94F42D0E94E8
:103AE000A51A0E946614823019F0833069F405C06B
:103AF00085E296E066E172E004C085E296E06FEF51
:103B000071E00E94FF2A08958FEF8093EF031092D7
:103B100056040E94FA190CC085E296E00E94BA2D64
:103B2000892B31F085E296E00E94F42D0E94A51ABF
:103B30008091EF038E3F81F708958091EF039927DD
:103B400087FD9095A92FB92FFC013196EB30F10537
:103B500008F074C0E254FF4F0C94672F85E296E0A2
:103B600064E678E00E94FF2A83E693E00E94C91988
:103B700085E296E06CE478E00E94FF2A85E296E018
:103B800067E278E00E94FF2A85E296E06DEF77E039
:103B90000E94FF2A85E296E06CED77E00E94FF2A02
:103BA00085E296E06FEA77E00E94FF2A85E296E0E0
:103BB00069E877E00E94FF2A85E296E065E677E013
:103BC0000E94FF2A85E296E06EE377E00E94FF2ADA
:103BD00085E296E00E94E92A0E94A2182FC085E2A1
:103BE00096E061E277E028C085E296E06CEF76E04F
:103BF00023C085E296E067EE76E01EC085E296E09F
:103C000068EC76E019C085E296E064E876E014C0DE
:103C100085E296E06FE676E00FC085E296E06AE521
:103C200076E00E94FF2A85E296E064E176E004C037
:103C300085E296E06EEF75E00E94FF2A6AE070E090
:103C400080E090E00E946E2904C085E296E00E9428
:103C5000F42D85E296E00E94BA2D892BB1F70895E4
:103C6000A2E2B0E0E6E3FEE10C94302F8E010F5F9C
:103C70001F4F80E1D8011D928A95E9F785E296E011
:103C800066EC71E00E94752C0E94121520E431EE62
:103C90004DE958E12F8F38A349A35AA380EC91ED49
:103CA000A8E9BBE18B8F9C8FAD8FBE8F24EF31E0F5
:103CB00040E050E02F8B388F498F5A8F60E5C62E39
:103CC00063ECD62EE12CF12C50E4452E51EE552E0E
:103CD0005DE9652E58E1752E88249924540133241A
:103CE0001E8A1D8A198A1A8A1B8A1C8AFFC085E2CD
:103CF00096E00E94F42D8434B9F0853430F4833298
:103D0000B9F18C3209F0CCC044C0833509F0C8C089
:103D10002F8D38A149A15AA1C901DA012C013D0119
:103D2000882499245401E2C085E296E064E40E946C
:103D3000E12A85E296E040E451EE6DE978E12AE07F
:103D400030E00E94152C85E296E06CE20E94E12AA8
:103D500085E296E040EC51ED68E97BE12AE030E055
:103D60000E94152C85E296E06CE20E94132BBEC0E7
:103D700019821A821B821C821D821E821F82188653
:103D800019861A861B861C861D861E861F86188A23
:103D90003AC0339434E0331609F0A8C069817A81BF
:103DA0008B819C8128EE33E040E050E00E94C12EE0
:103DB0006F8F78A389A39AA36D817E818F81988567
:103DC0000E94C12E6B8F7C8F8D8F9E8F89859A85E7
:103DD000AB85BC858F8B988FA98FBA8F6D857E85BB
:103DE0008F8598890E94C12E6B017C0190E2C916D3
:103DF0009EE4D90690E0E90690E0F90630F48CE103
:103E000062E30E94B50A332471C0A0E3CA16A5E795
:103E1000DA06A0E0EA06A0E0FA0618F48CE162E215
:103E2000F0CFB0E4CB16BCE9DB06B0E0EB06B0E0C7
:103E3000FB0618F48CE166E2E4CFE0E5CE16E3EC95
:103E4000DE06E0E0EE06E0E0FE0618F48CE162E15A
:103E5000D8CFF0E6CF16FAEEDF06F0E0EF06F0E09E
:103E6000FF0618F48CE165E1CCCF20E7C21621E112
:103E7000D20621E0E20620E0F20618F48CE161E0CF
:103E8000C0CF30EAC31636E8D30631E0E30630E0AF
:103E9000F30618F48CE163E0B4CF8CE165E0B1CFB8
:103EA00040ED242E280E49E0421500F1032D10E0CC
:103EB000000F111F000F111F81E090E08C0F9D1F5C
:103EC000080F191FD8016D917D918D919C912AE069
:103ED00030E040E050E00E94C12E620D711D811D56
:103EE000911DF801608371838283938385E296E05C
:103EF0000E94BA2D892B09F0FACE81149104A104F5
:103F0000B10489F4C301B2010E942B0B61E070E09F
:103F100080E090E00E946E29FFEFFE8B1D8A198AD7
:103F20001A8A1B8A1C8A2F89388D498D5A8D8216D0
:103F30009306A406B506E0F40E94D60A29893A89B8
:103F40004B895C89280F311D411D511D298B3A8BEE
:103F50004B8B5C8B3D89381708F48D8B4E89841709
:103F600008F48E8B0894811C911CA11CB11C56C0B6
:103F7000C301B20128EE33E040E050E00E94F32E8E
:103F800085E296E0BA01A9012AE030E00E94A72B61
:103F900085E296E06CE20E94E12A85E296E06D8976
:103FA0004AE050E00E94EF2B85E296E06CE20E942E
:103FB000E12A69897A898B899C89A50194010E94EB
:103FC000F32E85E296E0BA01A9012AE030E00E94D2
:103FD000A72B85E296E06CE20E94E12A85E296E05A
:103FE0006E894AE050E00E94EF2B85E296E06CE299
:103FF0000E94132B4C0C5D1C6E1C7F1C8B8D9C8DAA
:10400000AD8DBE8D84159505A605B70520F44F8CA2
:1040100058A069A07AA08824992454012F8D38A132
:1040200049A15AA1285E33404040504009F05ECF7C
:10403000A296E2E10C944C2FAAE5B0E0E2E2F0E2B5
:104040000C943C2F8B017A018B3009F425C18C3004
:1040500040F5853009F484C0863080F4823009F45C
:1040600059C0833020F4813009F058C242C08330F7
:1040700009F461C0843009F051C265C0883009F488
:104080009DC0893038F4863009F486C0873009F045
:1040900045C28CC0893009F499C08A3009F03EC20B
:1040A000C9C0893609F48AC18A3680F4863609F493
:1040B00035C1873620F4853609F030C216C18736FF
:1040C00009F445C1883609F029C249C18C3609F482
:1040D000CCC18D3638F48A3609F47BC18B3609F0B1
:1040E0001DC2B7C18D3609F4F4C1873C09F016C270
:1040F00008C281E069E270E00E945B110EEB13E000
:10410000F80181918F010E944411F3E0073E1F07DF
:10411000B9F70CC282E06BE170E00E945B1103EA28
:1041200013E0F80181918F010E944411F3E00E3BEE
:104130001F07B9F7FBC183E061E070E00E945B11EB
:104140000E946614F1C184E061E070E00E945B119E
:1041500081E00E9444110E943D110E94301EE8C17E
:104160006091770470E0660F771F85E00E945B1115
:1041700000E010E008C0F801E95AFB4F80810E947E
:1041800044110F5F1F4F8091770490E0880F991FB3
:104190000817190780F3CAC186E062E070E00E9448
:1041A0005B1183E693E00E945211C0C187E061E099
:1041B00070E00E945B1180917804B6C188E061E0F4
:1041C00070E00E945B1180919903AEC186E68983FD
:1041D000CE01019661E00E94A30F0E94740C83E05F
:1041E0008093980368EC70E080E090E00E946E2974
:1041F000809198038430E1F48FE70E948B0A0E943B
:104200009F0A8983863471F489E060E270E00E943D
:104210005B1110E00E949F0A0E9444111F5F103240
:10422000C9F784C189E061E070E00E945B11CFC0F2
:1042300089E075C18AE069E070E00E945B1110922C
:104240009A0380918F05882351F080919F0390916C
:10425000A003A091A103B091A203806809C080913E
:104260009F039091A003A091A103B091A2038F7727
:1042700080939F039093A003A093A103B093A20304
:104280000AE913E0F80181918F010E944411F3E0E3
:10429000033A1F07B9F74AC18BE061E270E00E9460
:1042A0005B118091AC048F3F39F08091AC048F5F3B
:1042B0008093AC04815002C08091AC040E944411F0
:1042C00000E010E0F894F801EE0FFF1FE95DFC4FED
:1042D000808191810E940E0A0E94521178940F5F92
:1042E0001F4F0031110571F721C185E661E070E0D3
:1042F0000E945B110932110509F015C120E030E080
:10430000F901E254FC4FD701A20FB31F8C918083B7
:104310002F5F3F4F2932310599F759C086E661E09A
:1043200070E00E945B110B31110509F0FCC020E028
:1043300030E0F901ED55FC4FD701A20FB31F8C916E
:1043400080832F5F3F4F2B31310599F740C087E6BF
:1043500061E070E00E945B110E94111638C088E68F
:1043600061E070E00E945B1185E78A83DE011396AD
:10437000E3EAF3E08BE101900D928150E1F7CE0189
:1043800002966CE10E94A30F0E94740C83E080935C
:10439000980360E273E080E090E00E946E298091D3
:1043A0009803843009F0BFC08FE70E948B0A0E94F7
:1043B0009F0A8A83853509F0B6C009C089E661E0A5
:1043C00070E00E945B110E944D080E94920881E0FB
:1043D000ABC08AE661E070E00E945B1189E68E8FD7
:1043E000CE014E9661E00E94A30F0E94740C83E000
:1043F0008093980360E273E080E090E00E946E2971
:1044000080919803843009F08EC08FE70E948B0A58
:104410000E949F0A8E8F8E01015E1F4F7AE3E72E66
:10442000F12CEC0EFD1E0E949F0AF80181938F0172
:10443000EE15FF05C1F7A3EAB3E0FE017F968BE11D
:1044400001900D928150E1F78E8D893409F06BC097
:10445000BECF8BE661E070E00E945B11F7018081C6
:104460000E943F160E941A16B2CF8CE661E070E0FF
:104470000E945B110032110571F487E68AAFDE01FC
:10448000DB96F70180E201900D928150E1F7CE01B9
:10449000CA9661E205C087E48AAFCE01CA9661E0A0
:1044A0000E94A30F0E94740C83E0809398036CE435
:1044B00074E080E090E00E946E298091980384303F
:1044C00091F58FE70E948B0A0E949F0A873459F565
:1044D0007ECF8DE661E070E00E945B11093011052E
:1044E00011F520E030E0F901E656FC4FD701A20FAC
:1044F000B31F8C9180832F5F3F4F2930310599F78F
:1045000066CF87EC61E070E00E945B1181E00E9461
:1045100044110E943D111092ED030AC08AEC61E043
:1045200070E00E945B1180E00E9444110E943D11E6
:10453000C65ADF4FE6E00C94582FA0E0B0E0E3EA63
:10454000F2E20C94382F54E0A52E46E0B42E35E06C
:10455000C32E03E215E024E6D22E92E0E92E83E09A
:10456000F82EA1C085E296E00E94F42D982F80934A
:104570008E0580918D05833021F1843028F48130BF
:1045800099F08230B8F409C0853009F448C085300C
:1045900020F1863009F087C05FC0953B09F083C0E9
:1045A00081E080938D057FC0923609F07AC0E09259
:1045B0008D0579C090938C0590938B05F0928D05B5
:1045C00072C09093890510928A0580918B05892786
:1045D00080938B05A0928D0566C0D92FC0E02091F5
:1045E000890530918A052C2B3D2B30938A05209329
:1045F000890580918B05892780938B05C0928D0555
:104600002536310508F44FC08CEC61E070E00E9463
:104610005B1181E00E9444110E943D1142C0209133
:10462000870530918805F901ED5DFA4F90838091FF
:104630008B05892780938B052F5F3F4F309388052B
:10464000209387058091890590918A05281739075D
:1046500050F1B0928D0527C080918B05891759F4D0
:10466000609187057091880580918C0543E255E043
:104670000E941C200DC08BEC62E070E00E945B1178
:1046800080918C050E9444118091EE030E94441198
:10469000F8018D2D11928A95E9F7109288051092F4
:1046A000870510928D0585E296E00E94BA2D892B30
:1046B00009F058CFCDB7DEB7EAE00C94542F81E073
:1046C0008093ED0308C085E296E00E94BA2D892B05
:1046D00011F00E949D228091ED038823A1F7089597
:1046E000A0E0B0E0E6E7F3E20C943B2F0E944829FB
:1046F0006115710581059105C9F30E949906109213
:10470000C7031092C8031092C9031092CA03DD2494
:10471000E090C703F090C8030091C9031091CA0349
:10472000102F0F2DFE2CEE240E9494062FEF30E068
:1047300040E050E00E94152FE60EF71E081F191FDB
:10474000E092C703F092C8030093C9031093CA0311
:10475000D39444E0D416E1F6CDECD3E000E010E0D1
:1047600060E1E62E67E2F62E4EC00F5F19F40E945C
:104770004D084DC00E94940622E330E040E050E036
:104780000E94152F6F5FEDECF3E090E004C0819183
:10479000861759F39F5F9117D0F38091CC0390E077
:1047A0008E9D90018F9D300D9E9D300D1124862F82
:1047B00090E0AC01249FC001259F900D349F900D87
:1047C0001124AA2797FDA095BA2F2091C3033091F9
:1047D000C4034091C5035091C603820F931FA41FC9
:1047E000B51F20919B0330919C0340919D035091F4
:1047F0009E03281739074A075B0708F4B6CF699369
:104800001F5F183121F08881882309F0AECFCDB722
:10481000DEB7E7E00C94572F1F931091EF031F3F73
:1048200009F0F1C0893409F467C08A3428F5883367
:1048300009F479C0893368F4803309F486C0813380
:1048400008F06FC08B3109F44DC0813209F0D5C03A
:104850003DC0813409F49AC0823438F4893309F4B4
:1048600072C0803409F0C9C031C0823409F4A1C0DB
:10487000863409F0C2C052C0823609F49AC0833629
:1048800090F4883579F1893538F4823509F43FC0E0
:10489000833509F0B2C01FC08A3509F4A9C081363A
:1048A00009F0ABC073C0823791F1833730F486369C
:1048B000A9F1893609F0A1C01FC0883799F08A375D
:1048C00009F496C0833709F098C005C085E296E0E8
:1048D00069E471E019C00E94111685E296E063ED6B
:1048E00071E006C00E941A1685E296E06DEE71E056
:1048F0000E94752C8EEF7FC00E944D080E94920886
:1049000085E296E06CE072E00E94752C76C00E9411
:10491000702385E296E065E272E0F6CF0E94C2164F
:104920006CC0805368C085E296E06CEE71E00E9436
:10493000FF2A9091E603892F885F8871977E892BE3
:104940008093E60320C089E056C085E296E069EDD9
:1049500071E00E94FF2A80919F039091A003A09193
:10496000A103B091A20320E130E040E050E08227B3
:104970009327A427B52780939F039093A003A09328
:10498000A103B093A2031093EF0337C085E296E032
:1049900063EC71E00E94FF2A80919F039091A00335
:1049A000A091A103B091A20320E430E040E050E0E8
:1049B00012C085E296E062EB71E00E94FF2A8091CE
:1049C0009F039091A003A091A103B091A20320E2C4
:1049D00030E040E050E082279327A427B52780935A
:1049E0009F039093A003A093A103B093A20302C0DE
:1049F0000E94591D8FEF8093EF038091EF038E3F4C
:104A000009F4DDC0D4C00E945916882309F4D7C028
:104A100080915504882321F48FEF8093EF03C7C062
:104A200080EF93E060E070E040E050E00E94A2067A
:104A30009B01AC018091EF03992787FD9095A92FE9
:104A4000B92FFC013197E930F10508F08CC0E7532C
:104A5000FF4F0C94672FDA01C9018154914EAD4983
:104A6000B8418F57904FAA4FB24008F07CC02093B6
:104A7000C3033093C4034093C5035093C6039AC045
:104A80002093C7033093C8034093C9035093CA03CC
:104A900081E0809356048EC02830310541055105D0
:104AA00008F061C02093CB0385C0DA01C9010197EA
:104AB000A109B1090A97A105B10508F054C02093D6
:104AC000CC0378C080EF93E06DE371E00E94BE07F5
:104AD00010E00EC0183130F4E12FF0E0E254FC4F4A
:104AE00087871F5F80E090E06DE371E00E94BE0762
:104AF000009759F00E94A007009761F706C0E12FC8
:104B0000F0E0E254FC4F17861F5F1831C0F352C02B
:104B1000253031054105510530F52093E5034AC0A4
:104B2000DA01C9010197A109B1090697A105B105EB
:104B3000D0F48091E603887F822B8093E6033AC00D
:104B4000DA01C9010197A109B1098050924CA14035
:104B5000B04048F42093BF033093C0034093C10397
:104B60005093C20327C085E296E068EA71E00E9494
:104B7000752C13C08091C7039091C803A091C903FD
:104B8000B091CA030196A11DB11D8093C7039093F4
:104B9000C803A093C903B093CA030E944F168FEFB6
:104BA0008093EF0385E296E06AE00E94132B0E9457
:104BB0009D1D05C0809156048823E1F2EECF1F9120
:104BC00008958FEF8093EF03109256040E949D1D6D
:104BD0000CC085E296E00E94BA2D892B31F085E267
:104BE00096E00E94F42D0E940C248091EF038E3FEA
:104BF00081F76AE070E080E090E00E946E2904C0D6
:104C000085E296E00E94F42D85E296E00E94BA2D9E
:104C1000892BB1F70895AAE2B0E0E1E1F6E20C9445
:104C2000352F0E943A297B018C0181E00E94950B6F
:104C300004C085E296E00E94F42D85E296E00E9491
:104C4000BA2D892BB1F75E984098DD24D394A2E663
:104C50007A2EF2E08F2E912C8C0E9D1E5E01089410
:104C6000A11CB11CE3E0CE2E0E943A2920E030E0E6
:104C70006E197F09800B910B693C710581059105C7
:104C800010F021E030E08D2D90E028233923232BF4
:104C9000A9F10E943A297B018C015D9A419A80ED2D
:104CA00097E00E948F117982D401EEEBF3E089E264
:104CB00001900D928150E1F7C5016AE20E94A30FB5
:104CC0005D98419880E090E00E948F11C092980317
:104CD0000E94740C62E370E080E090E00E946E2914
:104CE00080919803843051F4C09298038FE70E941A
:104CF0008B0A0E949F0A823409F4DD2483E10E941A
:104D00006C2A892B69F5DD24D3942AC05E9A409AD7
:104D10005D9A419A85E296E00E94F42D8D309105CE
:104D200069F08E3091051CF40A97B1F407C0833204
:104D3000910569F08234910579F40CC085E296E022
:104D400064EA71E00E94FF2A0E94E12505C00E94EA
:104D5000301E02C00E945F235E9840985D98419883
:104D600085E296E00E94BA2D892B09F47DCFCECF43
:104D70008F929F92AF92BF92CF92DF92EF92FF926B
:104D80000F931F9383E10E946C2A892B09F083C043
:104D900068EC70E080E090E00E946E2980E090E096
:104DA0000E948F110E943A295B016C01B0ECEB2E3E
:104DB000B2E1FB2E012D112DE60EF71E081F191F63
:104DC00006C083E10E946C2A892B09F062C00E9410
:104DD0003A296E157F058007910798F383E10E94B9
:104DE0006C2A892B09F055C080ED97E00E948F1145
:104DF0000E943A297B018C0199249394882488E4A9
:104E000096E2A0E0B0E0A80EB91ECA1EDB1E29C0C3
:104E1000AE14BF04C006D10638F480ED97E00E94BE
:104E20008F11882483941DC00E943A296E197F092E
:104E3000800B910B693C71058105910590F00E94F2
:104E40003A297B018C0180E0992009F481E0982EB9
:104E5000882319F480E090E002C080ED97E00E9482
:104E60008F1183E10E946C2A892B91F280E090E0FF
:104E70000E948F11882049F0809199038F5F837081
:104E80000E943F160E941A1606C00E9470230E94BC
:104E900011160E940B261F910F91FF90EF90DF904B
:104EA000CF90BF90AF909F908F90089580E06DEF6E
:104EB00077E042E050E00E9475280895EF92FF925B
:104EC0000F931F9380E00E9419080E947A1186E0D8
:104ED00061E00E94CD2985E061E00E94CD298EE04D
:104EE00061E00E94CD298FE061E00E94CD2983E13D
:104EF00060E00E94CD2988E060E00E94CD2988E032
:104F000061E00E94392A0E943E1485E296E040E06A
:104F100052EC61E070E00E94332D0E9432160E9434
:104F20001A160E94390D8FEF8093AC040E94562709
:104F300078940E943A297B018C018091AC048F3FC8
:104F400009F0C8C00E943A296E197F09800B910BA5
:104F5000605D77408040904008F0BCC0EECF85E2B5
:104F600096E00E94F42D85E296E00E94BA2D892BEE
:104F7000B1F785E296E062E472E00E94722C83E66B
:104F800093E00E94C91985E296E069E572E00E940B
:104F9000722C85E296E067E070E04AE050E00E9403
:104FA0005E2C62E370E080E090E00E946E2985E272
:104FB00096E00E94BA2D04970CF185E296E00E94DB
:104FC000F42D82349105D1F485E296E00E94F42D0F
:104FD0008E34910599F485E296E00E94F42D843494
:104FE000910561F485E296E00E94F42D819731F4F9
:104FF00080E090E00E948F110E940B264091BF0339
:105000005091C0036091C1037091C203DB01CA01DA
:105010000197A109B1090497A105B10568F440936E
:10502000AD04433029F040E052EC61E070E004C090
:1050300040EA56E861E070E085E296E00E94332D98
:105040000E94B8265E98409880E090E00E948F1100
:105050000E94390D80E00E94950B809192040E947D
:10506000C00A0E94740C1092170510921805109235
:10507000190510E015C062E370E080E090E00E9446
:105080006E2980ED97E00E948F1162E370E080E06E
:1050900090E00E946E2980E090E00E948F111F5FD7
:1050A00080919903811738F78091E60390E084FF9F
:1050B00009C020E088719070489709F421E0822FA0
:1050C0000E9447148FE00E9419081F910F91FF90D2
:1050D000EF90089580ED97E00E948F1183E161E0E9
:1050E0000E94392A5E9A409A3ECF823000F5E82F1E
:1050F000F0E0EE0FFF1FE057FA4F718360838823C3
:1051000019F08130A1F408C0809169008C7F842B54
:1051100080936900E89A089580916900440F551FB3
:10512000440F551F837F842B80936900E99A08956B
:105130001F920F920FB60F9211242F933F934F930C
:105140005F936F937F938F939F93AF93BF93EF93EF
:10515000FF938091900590919105892B29F0E09122
:105160009005F09191050995FF91EF91BF91AF9155
:105170009F918F917F916F915F914F913F912F916F
:105180000F900FBE0F901F9018951F920F920FB6A1
:105190000F9211242F933F934F935F936F937F93BD
:1051A0008F939F93AF93BF93EF93FF93809192055B
:1051B00090919305892B29F0E0919205F091930548
:1051C0000995FF91EF91BF91AF919F918F917F9141
:1051D0006F915F914F913F912F910F900FBE0F9064
:1051E0001F9018951F920F920FB60F9211242F93B4
:1051F0003F938F939F93AF93BF9380919805909126
:105200009905A0919A05B0919B0530919C05019656
:10521000A11DB11D232F2D5F2D3720F02D57019695
:10522000A11DB11D20939C0580939805909399052D
:10523000A0939A05B0939B05809194059091950554
:10524000A0919605B09197050196A11DB11D80937F
:10525000940590939505A0939605B0939705BF91FB
:10526000AF919F918F913F912F910F900FBE0F9013
:105270001F9018958FB7F894209198053091990553
:1052800040919A0550919B058FBFB901CA010895BD
:105290009FB7F8942091940530919505409196051B
:1052A0005091970586B5A89B06C08F3F21F02F5FD0
:1052B0003F4F4F4F5F4F9FBF542F432F322F222717
:1052C000280F311D411D511D82E0220F331F441F45
:1052D000551F8A95D1F7B901CA010895EF92FF923F
:1052E0000F931F93CF93DF937B018C010E9448297A
:1052F000EB010EC00E9448296C1B7D0B685E734059
:10530000C8F30894E108F10801091109C851DC4FFC
:10531000E114F1040105110569F7CDB7DEB7E6E048
:105320000C94582F789484B5826084BD84B58160D4
:1053300084BD85B5826085BD85B5816085BDEEE69D
:10534000F0E0808181608083E1E8F0E0108280817C
:1053500082608083808181608083E0E8F0E08081EA
:1053600081608083E1EBF0E0808184608083E0EB0A
:10537000F0E0808181608083EAE7F0E080818460F2
:10538000808380818260808380818160808380814E
:10539000806880831092C1000895CF93DF93482FD7
:1053A00050E0CA018D5F934FFC0134914151544F3D
:1053B000FA018491882369F190E0880F991FFC011C
:1053C000EF52F44FA591B491FC01E552F44FC59111
:1053D000D491662351F42FB7F8948C91932F909524
:1053E00089238C93888189230BC0623061F42FB7A5
:1053F000F8948C91932F909589238C938881832B9B
:1054000088832FBF06C09FB7F8948C91832B8C9311
:105410009FBFDF91CF910895833071F0843028F4DD
:105420008130A1F0823021F514C08630B1F0873090
:10543000D1F08430E9F404C0809180008F7703C0FC
:10544000809180008F7D80938000089584B58F7750
:1054500002C084B58F7D84BD08958091B0008F77A0
:105460008093B00008958091B0008F7D8093B0004C
:105470000895FF920F931F93F62E482F50E0CA0114
:10548000895E934FFC012491CA018D5F934FFC010B
:1054900014914151544FFA0104910023C9F0222381
:1054A00019F0822F0E940C2AE02FF0E0EE0FFF1F70
:1054B000E552F44FA591B4919FB7F894FF2021F4E1
:1054C0008C911095812302C08C91812B8C939FBF6E
:1054D0001F910F91FF9008950F931F93482F50E055
:1054E000CA01895E934FFC012491CA018D5F934FDD
:1054F000FC0104914151544FFA011491112319F404
:1055000020E030E015C0222319F0822F0E940C2ADF
:10551000812F90E0880F991F8B51944FFC01A5912A
:10552000B4918C9120E030E0802311F021E030E054
:10553000C9011F910F910895A0E0B0E0E2EAFAE2FC
:105540000C943A2F7C016B018A01C0E0D0E00FC0BF
:10555000D6016D916D01D701ED91FC910190F08123
:10556000E02DC7010995C80FD91F01501040011542
:10557000110571F7CE01CDB7DEB7E8E00C94562FD8
:10558000EF92FF920F931F93CF93DF937C018B01D8
:10559000C0E0D0E0F8010F5F1F4F6491662359F01F
:1055A000D701ED91FC910190F081E02DC7010995A3
:1055B000C80FD91FEFCFCE01CDB7DEB7E6E00C9410
:1055C000582FDC01ED91FC910190F081E02D0995BF
:1055D0000895EF92FF920F931F938C016DE00E944C
:1055E000E12A7C01C8016AE00E94E12A9C012E0D9B
:1055F0003F1DC9011F910F91FF90EF900895EF9209
:10560000FF920F931F937C010E94C02A8C01C70157
:105610000E94E92A9C01200F311FC9011F910F919F
:10562000FF90EF900895EF92FF920F931F937C01EC
:105630000E94E12A8C01C7010E94E92A9C01200FE7
:10564000311FC9011F910F91FF90EF900895CF93E3
:10565000DF93EC016115710519F420E030E00FC013
:10566000DB010D900020E9F71197A61BB70BE8812D
:10567000F9810280F381E02DAD0109959C01C901FA
:10568000DF91CF9108954F925F927F928F929F9278
:10569000AF92BF92CF92DF92EF92FF920F931F9340
:1056A000DF93CF93CDB7DEB7A1970FB6F894DEBFE7
:1056B0000FBECDBF2C01742ECB01223008F42AE09E
:1056C00019A231E2C32ED12CCC0EDD1E822E9924DC
:1056D000AA24BB24672D752FA50194010E94F32EE7
:1056E00079018A01C801B701A50194010E94C12E68
:1056F000472D461B0894C108D1084A3010F4405D7C
:1057000001C0495CF6014083E114F1040105110573
:1057100021F07E2C5F2DC801DDCFC201B6010E94B1
:10572000272BA1960FB6F894DEBF0FBECDBFCF9149
:10573000DF911F910F91FF90EF90DF90CF90BF907E
:10574000AF909F908F907F905F904F900895DC0175
:105750002115310541F4ED91FC910190F081E02D8E
:10576000642F099508950E94432B0895EF92FF92AC
:105770000F931F937C010E94A72B8C01C7010E94ED
:10578000E92A9C01200F311FC9011F910F91FF9041
:10579000EF900895EF92FF920F931F939A017B0170
:1057A00000E010E0B801A7010E94A72B1F910F9104
:1057B000FF90EF900895EF92FF920F931F937C015B
:1057C0000E94CA2B8C01C7010E94E92A9C01200F6C
:1057D000311FC9011F910F91FF90EF900895EF9233
:1057E000FF920F931F939A01E62EFF2400E010E032
:1057F000B801A7010E94A72B1F910F91FF90EF9076
:105800000895EF92FF920F931F937C010E94EF2B5C
:105810008C01C7010E94E92A9C01200F311FC90198
:105820001F910F91FF90EF900895A0E0B0E0EBE1A1
:10583000FCE20C943A2FEC016A017B012115310541
:1058400041F4E881F9810190F081E02D642F099500
:105850001BC02A303105B1F477FF13C06DE20E94FE
:10586000E12A8C0144275527BA014C195D096E09BC
:105870007F09CE012AE00E94432B9C01200F311F9B
:1058800004C02AE00E94432B9C01C901CDB7DEB7BA
:10589000E8E00C94562FEF92FF920F931F937B0139
:1058A0009A010027F7FC0095102FB801A7010E946C
:1058B000152C1F910F91FF90EF900895EF92FF929A
:1058C0000F931F937C010E944B2C8C01C7010E94F7
:1058D000E92A9C01200F311FC9011F910F91FF90F0
:1058E000EF9008950E94272B0895EF92FF920F9357
:1058F0001F937C010E94722C8C01C7010E94E92A2F
:105900009C01200F311FC9011F910F91FF90EF9053
:10591000089508951F920F920FB60F9211242F939E
:105920003F934F938F939F93EF93FF938091C0008A
:1059300082FD1DC04091C6002091DD053091DE053D
:105940002F5F3F4F2F7330708091DF059091E005FE
:105950002817390771F0E091DD05F091DE05E35677
:10596000FA4F40833093DE052093DD0502C080911D
:10597000C600FF91EF919F918F914F913F912F9191
:105980000F900FBE0F901F9018951F920F920FB699
:105990000F9211242F933F938F939F93EF93FF9335
:1059A00020912106309122068091230690912406B1
:1059B0002817390731F48091C1008F7D8093C10091
:1059C00014C0E0912306F0912406EF51FA4F208194
:1059D000809123069091240601968F739070909386
:1059E0002406809323062093C600FF91EF919F9198
:1059F0008F913F912F910F900FBE0F901F90189590
:105A0000A0E0B0E0E6E0FDE20C94362FFC0113824A
:105A1000128288EE93E0A0E0B0E084839583A683B1
:105A2000B7838AE893E0918380837587648757877B
:105A30004687318B208B138B028BF58AE48AD78AB9
:105A4000C68AB18EA08E938E828E8F85848F888930
:105A5000858F8989868F8A89878F8B8980A32096F5
:105A6000ECE00C94522FAF92BF92DF92EF92FF9234
:105A70000F931F93CF93DF93EC017A018B01DD2409
:105A8000403081EE580780E0680780E0780711F029
:105A9000DD24D39491E0A92EB12CEC89FD89DD2081
:105AA00069F0C50108A002C0880F991F0A94E2F7A7
:105AB000808360E079E08DE390E005C0108260E8CB
:105AC00074E88EE190E0A80197010E94F32E215026
:105AD000304040405040569547953795279580E196
:105AE0002030380720F0DD2011F0DD24D6CFE88902
:105AF000F9893083EA89FB89208319A2EE89FF891D
:105B0000408121E030E0C9010C8C02C0880F991F50
:105B10000A94E2F7482B4083EE89FF894081C9014E
:105B20000D8C02C0880F991F0A94E2F7482B40831E
:105B3000EE89FF894081C9010E8C02C0880F991F30
:105B40000A94E2F7482B4083EE89FF8980810F8C0D
:105B500002C0220F331F0A94E2F7209528232083E6
:105B6000DF91CF911F910F91FF90EF90DF90BF9049
:105B7000AF900895DC011C96ED91FC911D97E05CBF
:105B8000FF4F2191319180819181281B390B2F7317
:105B90003070C901089585E296E00E94BA2D892BE4
:105BA00011F00E94892C0895DC011C96ED91FC9166
:105BB0001D97E05CFF4F20813181E054F040DF0110
:105BC000AE5BBF4F8D919C9111972817390719F43F
:105BD0002FEF3FEF07C08D919C91E80FF91F808157
:105BE000282F30E0C9010895DC011C96ED91FC914D
:105BF0001D97E05CFF4F20813181E054F040DF01D0
:105C0000AE5BBF4F8D919C9111972817390719F4FE
:105C10002FEF3FEF10C08D919C911197E80FF91F66
:105C200020818D919C91119701968F7390701196A0
:105C30009C938E9330E0C9010895DC0191968C917C
:105C40009197882339F05496ED91FC915597808176
:105C500086FFF9CF91961C920895CF93DF93EC01C4
:105C6000EE85FF85E05CFF4F20813181E054F040FC
:105C70002F5F3F4F2F733070DF01AE5BBF4F8D91B1
:105C80009C91119728173907D1F3E05CFF4F808171
:105C90009181E054F040E80FF91F6083EE85FF85A5
:105CA000E05CFF4F31832083EE89FF89208181E012
:105CB00090E00F8C02C0880F991F0A94E2F7282BFE
:105CC000208381E089A3EC89FD89808180648083C1
:105CD00081E090E0DF91CF9108958F929F92AF92F3
:105CE000BF92CF92DF92EF92FF920F931F9300D05B
:105CF00000D00F92EDB7FEB7319684E0ADB7BEB7D6
:105D000011968C9383E0818387E0828385E083838F
:105D100081E0848385E296E06DE975E041EE55E02F
:105D200025EC30E004EC10E0B0ECEB2EF12CA1EC13
:105D3000CA2ED12CF2ECAF2EB12CE6EC8E2E912C8B
:105D40000E94002D0F900F900F900F900F901F91B9
:105D50000F91FF90EF90DF90CF90BF90AF909F900A
:105D60008F900895CF93DF930E9492290E945E271F
:105D7000CBECDDE20E9499112097E1F30E94CB2D3C
:105D8000F9CF629FD001739FF001829FE00DF11D5A
:105D9000649FE00DF11D929FF00D839FF00D749FA5
:105DA000F00D659FF00D9927729FB00DE11DF91F51
:105DB000639FB00DE11DF91FBD01CF0111240895AE
:105DC00097FB092E07260AD077FD04D086D006D08F
:105DD00000201AF4709561957F4F0895F6F790951D
:105DE00081959F4F0895A1E21A2EAA1BBB1BFD01AE
:105DF0000DC0AA1FBB1FEE1FFF1FA217B307E407AA
:105E0000F50720F0A21BB30BE40BF50B661F771F01
:105E1000881F991F1A9469F76095709580959095E1
:105E20009B01AC01BD01CF01089597FB092E05260A
:105E30000ED057FD04D0D7DF0AD0001C38F450959F
:105E40004095309521953F4F4F4F5F4F0895F6F79E
:105E500090958095709561957F4F8F4F9F4F0895D6
:105E60002F923F924F925F926F927F928F929F926A
:105E7000AF92BF92CF92DF92EF92FF920F931F9358
:105E8000CF93DF93CDB7DEB7CA1BDB0B0FB6F89409
:105E9000DEBF0FBECDBF09942A88398848885F8449
:105EA0006E847D848C849B84AA84B984C884DF80BA
:105EB000EE80FD800C811B81AA81B981CE0FD11D9E
:105EC0000FB6F894DEBF0FBECDBFED010895EE0F03
:105ED000FF1F0590F491E02D0994AA1BBB1B51E113
:105EE00007C0AA1FBB1FA617B70710F0A61BB70B4A
:105EF000881F991F5A95A9F780959095BC01CD01EF
:105F00000895911106C0803219F089508550D0F75C
:0C5F10000895992788270895F894FFCF82
:105F1C004E6F005965730054582074696D656F7528
:105F2C007421006D6F64756C65206C6F636B6564B8
:105F3C003F00486F70206368616E6E656C200020B6
:105F4C0040200053004E2F4100386368002C002C79
:105F5C00205B005D20280029004E4F5420454E4107
:105F6C00424C45440053656E64696E6720736574DA
:105F7C0074696E677320746F2052580A00526573EF
:105F8C00657474696E672073657474696E677320C9
:105F9C006F6E2052580A0041626F727465642065FE
:105FAC00646974730A00696E76616C696420736548
:105FBC006C656374696F6E000D0A496E76616C696D
:105FCC006420696E707574202D206469736361722E
:105FDC006465642107007363616E6E6572206D6F7A
:105FEC0064650053657474696E67732073617665BC
:105FFC006420746F20454550524F4D0A005265760F
:10600C0065727465642073657474696E6773206659
:10601C00726F6D20454550524F4D0A004C6F6164B4
:10602C00656420666163746F72792064656661755E
:10603C006C74730A004B657920616E64206368612F
:10604C006E6E656C732072616E646F6D697A6564D7
:10605C000A004F70656E4C52536E67205458207373
:10606C0074617274696E672000206F6E204857202F
:10607C000050504D00525353490053444100534378
:10608C004C00525844005458440041494E004C4274
:10609C004545500053504B54524D005342555300FC
:1060AC0053554D44004C4C494E440000342B3400A5
:1060BC003800382B340031320031322B3400313679
:1060CC000001000000C01200001A400AA1204EA5D9
:1060DC00001B1E27522C23308025000005400AA1EE
:1060EC00204EA50020244EA52C2330004B0000068A
:1060FC00400AD0009D49007B289D492C233000E1AB
:10610C00000005400A4501D7DC03B81E0EBF002372
:10611C002E48E801008A400A6001555502AD1E2048
:10612C00000023C88025000005400AA1204EA500D0
:10613C0020244EA52C233000020002000200020095
:10614C000200020002000200020002000200020033
:10615C0002000200020002FF610265026A026E0286
:10616C00720276027A027E0284028B0290029502FF
:10617C009B029B029B029B0235019C02A002A20285
:10618C00A602A902AE02350100070B0C1011150076
:10619C00160A13223129000000002D2E9C2ABA2D3C
:0661AC00F42DD42D1D2E80
:00000001FF
